:1000000012C017C016C015C014C013C012C011C052
:1000100010C00FC00EC00DC00CC00BC00AC009C07C
:1000200008C007C006C011241FBECFEDCDBF66D0EB
:100030009CC0E6CF282F392FC90102C000000197CC
:1000400018161906DCF3089598B321E030E002C0D9
:10005000220F331F8A95E2F72095292328BBCB0175
:10006000E9DF089598B321E030E002C0220F331F8A
:100070008A95E2F7922B98BBCB01DCDF0895EF92D3
:10008000FF920F931F93CF93DF938C01C0E0D0E0DA
:100090008CEDE82E85E0F82EC801BE01E3DFB70144
:1000A0006C1B7D0BC801D0DF219685E0CC3DD807C5
:1000B00099F7DF91CF911F910F91FF90EF900895E5
:1000C000EF92FF920F931F93CF93DF938C01CCEDB0
:1000D000D5E09CEDE92E95E0F92EC801BE01C2DF06
:1000E000B7016C1B7D0BC801AFDF2197B1F7DF9122
:1000F000CF911F910F91FF90EF900895B89AB99A00
:10010000BA9AB09AB19AB29A80E090E060E070E05A
:10011000A9DF81E090E0B3DF81E090E060E070E093
:10012000A1DF80E090E0CCDF81E090E060E070E073
:1001300099DF82E090E0A3DF82E090E060E070E091
:1001400091DF81E090E0BCDF82E090E060E070E071
:1001500089DF80E090E093DF80E090E060E070E095
:0E01600081DF82E090E0ACDFCFCFF894FFCFDC
:00000001FF
